:107C0000112484B714BE81FF05D185E080938100E3
:107C100082E08093C00088E18093C10086E0809379
:107C2000C20080E18093C4008EE0DED0259A86E019
:107C300020E33CEF91E0309385002093840096BBD5
:107C4000B09BFECF1D9AA8958150A9F7CC24DD24C6
:107C5000AA24A394B5E09B2EA1E18A2EF3E0BF2EC7
:107C6000B7D0813409F5B4D0082FC4D0023811F050
:107C7000013811F484E016C0003A11F483E112C017
:107C8000013A11F484E50EC0023A11F480E10AC011
:107C9000033A39F49DD08093C4009AD08132E9F739
:107CA0008CC083E08DD089C0823411F484E103C09C
:107CB000853419F485E0A6D080C0853579F488D064
:107CC000E82EFF2485D0082F10E0102F00270E2962
:107CD0001F29000F111F8ED068016FC0863521F457
:107CE00084E090D080E0DECF843609F040C070D0D0
:107CF0006FD0082F6DD080E0C81680E7D80618F442
:107D0000F601B7BEE895C0E0D1E062D089930C17C8
:107D1000E1F7F0E0CF16F0E7DF0618F0F601B7BEA6
:107D2000E89568D007B600FCFDCFA601A0E0B1E061
:107D30002C9130E011968C91119790E0982F882724
:107D4000822B932B1296FA010C01A7BEE895112401
:107D50004E5F5F4FF1E0A038BF0751F7F60197BEC5
:107D6000E89507B600FCFDCF87BEE89526C08437AE
:107D7000B1F42ED02DD0F82E2BD03CD0F601EF2C24
:107D80008F010F5F1F4F84911BD0EA94F801C1F758
:107D90000894C11CD11CFA94CF0CD11C0EC085379D
:107DA00039F428D08EE10CD085E90AD08FE07ACF63
:107DB000813511F488E018D01DD080E101D050CF7A
:107DC000982F8091C00085FFFCCF9093C600089546
:107DD0008091C00087FFFCCF8091C00084FD01C06E
:107DE000A8958091C6000895E0E6F0E098E19083C0
:107DF00080830895EDDF803219F088E0F5DFFFCF52
:107E000084E1DECF1F93182FE3DF1150E9F7F2DF93
:0E7E10001F91089580E0E8DFEE27FF27099418
:027FFE00040479
:0400000300007C007D
:00000001FF
